:1000000000F00CEF00F0E803FFFFF9EF0FF00A003B
:10001800FFFF00EEA7F0590EEE6AE806FDE10E6A52
:100028000D6A05EE68F08E0EEE6AE806FDE105EE53
:0800380067F00E0EF66E000EDB
:10004000F76E0900F5CFEEFF00EEF5F0060EF66E46
:10005000000EF76E10EE02F00900F5CFEEFFE5504E
:10006000E150FAE1E25002E02CEF00F098EF0CF0E2
:10007000026A016A006AE950EA1006E002C0EDFF78
:1000800001C0EDFF00C0EFFF000CFFFFD10EE16EDD
:10009000050EE26ED96A200EE76EE652D92A1F0ECF
:1000A000D964F9D71200FFFFF1D7FB00FFFFE16E23
:1000B000200EE1604CD0D10EE124D96EDA6A050E33
:1000C000DA2230D0FBC0F6FFFCC0F7FF050EF76464
:1000D00004D00800FFFFF55005D0F6CFE9FFF7CFB9
:1000E000EAFFEF50090A19E00001FD5105E00501A2
:1000F00070A702D0200E10D0FBC0F6FFFCC0F7FFA7
:10010000050EF76404D00800FFFFF55005D0F6CFC8
:10011000E9FFF7CFEAFFEF50DF6EDE520001FB4B45
:10012000FC2BE12AFBC0F6FFFCC0F7FF050EF764CD
:1001300004D00800FFFFF55005D0F6CFE9FFF7CF58
:10014000EAFFEF50000903E01F0EE164BBD7120085
:10015000FFFFADD7F700FFFFD96E200ED96008D0A2
:10016000D95005EED1F0E926000EEA22F7C0EFFFE4
:100170001200FFFFF1D7FB00FFFFD96E0001FD5118
:10018000FC1128E1D10ED924E16EE26A050EE222CB
:1001900013D00001FF510CE0050170A709D0E1CF99
:1001A000D9FFE2CFDAFFE14AE22A200EDF6E02D069
:1001B000FEC0E6FF0001FB07020EFB61EAD700016B
:1001C000FF5106E0050170A703D0200EE76E8FD027
:1001D000300EFCD7D950FBC000F0016A0026000E9B
:1001E0000122D10E0024E16E050E0120E26E000115
:1001F000FF511EE00501FF0EE106E222E1CFD9FF2B
:10020000E2CFDAFF70A71BD0200EDF6E020E0001D6
:100210000CD0FF0EE106E222E1CFD9FFE2CFDAFFF8
:10022000200EDF6E0001FB07020EFB61F2D75FD0EC
:10023000FF0EE106E222E1CFD9FFE2CFDAFF0A0E9C
:10024000026E036AFCC000F0FDC001F0C8EC02F0D1
:100250000050300FDF6E0A0EF66EF76A020E0001D4
:1002600044D0F6CF02F0F7CF03F0FCC000F0FDC0A1
:1002700001F0C8EC02F0055004101EE0FF0EE1068C
:10028000E222E1CFD9FFE2CFDAFFF6CF02F0F7CFDB
:1002900003F0FCC000F0FDC001F0C8EC02F004C0A7
:1002A00000F005C001F00A0E026E036AC8EC02F00D
:1002B0000050300FDF6E09D0FF0EE106E222E1CFE1
:1002C000D9FFE2CFDAFFFEC0DFFF0A0E026E036A3B
:1002D000F6CF00F0F7CF01F0FAEC12F004C0F6FF11
:1002E00005C0F7FF0001FB07020EFB61BAD7120041
:1002F000FFFF43D7FFFF280ED96ED95002E0D90681
:10030000FCD71200FFFFF7D7F700FFFFF7C000F0A0
:10031000F8C001F0D89001320032D890013200329A
:1003200000C0F6FF01C0F7FFF36AF46AF750F45C0F
:1003300002E1F650F35C04E2DDDFF34AF42AF6D77B
:100340001200FFFFE3D7FFFFD96E0F0E8116D950C1
:10035000F00BE16EE15081128A848A940F0E8116AF
:10036000D938F00BF00BE16EE15081128A848A9447
:100370001200FFFFE9D7FFFF8A948A960F0E8116BD
:10038000E96AD890E934006E016A01360050E40F42
:10039000F66E0150F76E060EF7220900FFFFF5CF4B
:1003A000F7F00900FFFFF5CFF8F0AFDFE9CF00F07D
:1003B000016A0050F60FF66E0150F76E060EF72236
:1003C0000800FFFFF550BFDF00F0E92A080EE964DE
:1003D000D8D7F00E0001F76FF86B97DF0501709129
:1003E0001200FFFFC9D7FFFF8A96400EACDF0A0E4E
:1003F0000001F76FF86B89DFE96AE9CF00F0016A65
:100400000050FF0FF66E0150F76E060EF72208003F
:10041000FFFFF550F36E8A86F35095DF0A0E000158
:10042000F76FF86B72DFE92A1F0EE964E6D78A9648
:10043000800E89DF0A0E0001F76FF86B66D7FFFFA9
:10044000D3D7E96AEA6A0C6B086A096A0A6A0B6A16
:10045000045005100610071006E1046A056A066AD2
:10046000076AEAEF12F0C00E0C1606D0D8900436D8
:100470000536063607360C2A07AEF8D70C2AD89070
:10048000083609360A360B360750035C08E1065079
:10049000025C05E10550015C02E10450005C09E3E7
:1004A00008800450005E0550015A0650025A075059
:1004B000035AD89007320632053204320C060C502B
:1004C0003F0BDDE10CBC14EC13F00050046E015046
:1004D000056E0250066E0350076E0850006E0950FC
:1004E000016E0A50026E0B50036E0CAEEEEF12F06E
:1004F00014EC13F0EEEF12F0086A01340234066EC9
:1005000004E00836026A018E1200006A016A026A7B
:10051000000C089204340534076E05E0D8B0088258
:10052000056A048E1200076A036A046A056A1200EB
:1005300006480E840650E9E0019E08320630026E3D
:10054000D8B0018E3BEF00F0065220E0025010E0E0
:10055000020403E1002A01220222D8900232013271
:100560000032062AF1E10250EFE00EAA0E96F0D713
:100570000050011002100AE001BEDAD7062E02D0A8
:100580000E86DAD7D89000360136F6D738EF00F06D
:10059000066A046A056A0250031003E1006A016AF0
:1005A000000C1F0E0612D890062A02360336FCE312
:1005B000033202320250005C0350015804E3016E22
:1005C0000250005ED88004360536062E06BAF0D7F3
:1005D00006AE05D0041E042AD8B40506051F045033
:1005E000026E0550036E06AC000C001E002AD8B443
:0605F0000106011E000CD3
:10060000202020202020202020202020202020EF1B
:1006100020202020202020202020202020202020DA
:1006200020202020202020202020202020202020CA
:10063000A2B52020202020202020202020202020A3
:1006400041A042A1E045A3A4A5A64BA74D484FA8B1
:10065000504354A9AA58E1ABACE2ADAE62AFB0B121
:1006600061B2B3B4E365B6B7B8B9BABBBCBD6FBECF
:100670007063BF79E478E5C0C1E6C2C3C4C5C6C72C
:100680002211C00AC00AF8133411AA125011F8132B
:100690007A140016BE15B0157A140016BE15B015E2
:1006A0001E161E161E161E161E169214EE14C00AD4
:1006B0001E16CA14A61434161E16C00AC00AC00A92
:1006C0001E165415181590151E161E161E161E16EB
:1006D000C80A020B280EA60E860FC20FFC0F501080
:1006E000A810A00F3075F811F811F811F811F811D1
:1006F000F000F000F8113F3F3F2F28080C010600E2
:100700000000000000000000101014121F02040678
:1007100009090600000000080C0E0F0E0C0800DD91
:10072000CFD120322E3120762E20312E30362000AF
:10073000202020563D090902432FECE8ED2020201F
:10074000D23D09090902432020743D09093A0909EB
:100750002000543D090909024320202020200920BF
:10076000092000CDE0E3F0E5E220E4EE20090909EC
:100770000243200020C2FBE4E5F0E6EAE02009099C
:100780003A0909200003002000202020CEF1F2E0E9
:10079000EDEEE2E8F2FC3F2020282D2920CDE5F205
:1007A000202F20282B2920C4E000C7E0EAF0EEE942
:1007B000F2E52020EAE0ECE5F0F300CFF0EEF6E51C
:1007C000F1F120E7E0E2E5F0F8E5ED00CFF0EEE151
:1007D000EEE920F1E8ECE8F1F2EEF0E00020202074
:1007E0002020CEE1F0FBE22020202020202020202D
:1007F000F2E5F0ECEEEFE0F0FB20202020002020DE
:1008000020CDE5E8F1EFF0E0E2E5ED20202020202A
:1008100020F2E5F0ECEEF2F0E0EAF22020200020F9
:100820002020D2E0F0E8F0EEE2EAE02020202000F4
:100830002020202020543D09090243202020202090
:10084000002020202020543D0909090243202020B7
:1008500020004B66633D0909092020543D09090920
:1008600002430004002A000500284E29202D20EF15
:10087000F0EEF1ECEEF2F020CFF0E32E2020202875
:100880000129202D20EFF3F1EA20CFF0E32E2020E4
:1008900020284E29202D20EFF0EEF1ECEEF2F02092
:1008A000CFF0E32E00282D29202D20EFEE20EAEEB8
:1008B000ECEDE0F2EDEEE920F2E5ECEFE5F0E0F250
:1008C000F3F0E53B202020282B29202D20EFEE20DF
:1008D000E2FBF1EEEAEEE920F2E5ECEFE5F0E0F222
:1008E000F3F0E53B202020284E29202D20E2FBF5C7
:1008F000EEE43B202020282D29202D20EFEE20EAB9
:10090000EEECEDE0F2EDEEE920F2E5ECEFE5F0E003
:10091000F2F3F0E53B20202000C2E2E5E4E8F2E556
:1009200020EAEEECEDE0F2EDF3FE20F2E5ECEFE58F
:10093000F0E0F2F3F0F320282B292C282D29202D8C
:1009400020E8E7ECE5EDE8F2FC20F2E5ECEFE5F07D
:10095000E0F2F3F0F33B20280129202D20E2E2EE23
:10096000E420F2E5ECEFE5F0E0F2F3F0FB3B2028C9
:100970004E29202D20E2FBF5EEE43B20202020C272
:10098000E2E5E4E8F2E520EAEEECEDE0F2EDF3007A
:10099000C4EEE6E4E8F2E5F1FC20EDE0E3F0E5E2A8
:1009A000E020E4EE2032303002433B2020202020A3
:1009B0002020202020202020202020284E29202DEB
:1009C00020E2FBF5EEE43B20202020202020202008
:1009D000202020202020C4EEE6E4E8F2E5F1FC200F
:1009E000EDE0E3F0E5E200C2E2E5E4E8F2E520EA6A
:1009F000EEFDF4F4E8F6E8E5EDF220F2E5F0ECEED9
:100A0000EFE0F0FB20282B292C282D29202D20E891
:100A1000E7ECE5EDE8F2FC20EAEEFDF4F4E8F6E8B8
:100A2000E5EDF23B20280129202D20F1EEF5F0E044
:100A3000EDE8F2FC20EAEEFDF4F4E8F6E8E5EDF28C
:100A40003B20284E29202D20E2FBF5EEE43B202020
:100A50002020C2E2E5E4E8F2E520EAEEFDF4F4E865
:100A6000F6E8001F073007520763077407850787FA
:100A7000078907AA07BB07CC07DD07FE071F083059
:100A8000084108520863086508670800F700FFFF7F
:100A9000050188B112D005018881F9C0CBF0FAC0F8
:100AA000CCF0F9C0CFF0FAC0D0F0FBC0CDF0FCC064
:100AB000CEF0F7C0D3F0F8C0D4F01200FFFFE8D7B3
:100AC000FFFF1200FFFFFDD7FFFF630EF66E0A0E59
:100AD000F76E0900FFFFF5CFFBF00900FFFFF5CF30
:100AE000FCF00001FD6B000E56EC00F07FC500F03D
:100AF000690E00240001FB6FFC6B080E0ED3FFFF94
:100B0000E4D7FFFF650EF66E0A0EF76E0900FFFFD1
:100B1000F5CFFBF00900FFFFF5CFFCF00001FD6B06
:100B2000000E56EC00F0020E0001FB6F7CC5FCF0DD
:100B3000FD6B200EFE6F05017B53000ED8B4010E35
:100B40000001FF6F050EBCEC00F0030E0001FB6F0F
:100B500000EEFCF0DFC0EEFFE0C0EDFF200EFE6F08
:100B60007BC500F00004000ED8B4010EFF6F120E1A
:100B7000BCEC00F03C0E046E056A066A076AF1C020
:100B800000F0F2C001F0F3C002F0F4C003F021EC79
:100B900002F000C0F7F001C0F8F0020E0001FB6F98
:100BA0003C0E026E036AF7C000F0F8C001F0C8EC1A
:100BB00002F000C0FCF001C0FDF0300EFE6F7BC5FE
:100BC000E8FF030A000ED8B4010EFF6F1E0EBCEC46
:100BD00000F0020E0001FB6F3C0E026E036AF7C0CC
:100BE00000F0F8C001F0C8EC02F004C0FCF005C051
:100BF000FDF0300EFE6F7BC5E8FF020A000ED8B490
:100C0000010EFF6F6BD0FFFF7DD7FFFF650EF66E05
:100C10000A0EF76E0900FFFFF5CFFBF00900FFFF9A
:100C2000F5CFFCF00001FD6B000E56EC00F0020E5B
:100C30000001FB6F7CC5FCF0FD6B200EFE6FFF6BAF
:100C4000050EBCEC00F0030E0001FB6F00EEFCF0A3
:100C5000DFC0EEFFE0C0EDFF200EFE6FFF6B120E57
:100C6000BCEC00F03C0E046E056A066A076AF1C02F
:100C700000F0F2C001F0F3C002F0F4C003F021EC88
:100C800002F000C0F9F001C0FAF0020E0001FB6FA3
:100C90003C0E026E036AF9C000F0FAC001F0C8EC25
:100CA00002F000C0FCF001C0FDF0300EFE6FFF6BE3
:100CB0001E0EBCEC00F0020E0001FB6F3C0E026E3B
:100CC000036AF9C000F0FAC001F0C8EC02F004C0F9
:100CD000FCF005C0FDF0300EFE6FFF6B1B0EBCEF8D
:100CE00000F0FFFF93D7FFFF670EF66E0A0EF76E58
:100CF0000900FFFFF5CFFBF00900FFFFF5CFFCF087
:100D00000001FD6B000E56EC00F0030E0001FB6FBE
:100D100000EEFCF0DBC0EEFFDCC0EDFF200EFE6F4E
:100D2000FF6B020EBCEC00F06D0EF66E0A0EF76E55
:100D30000900FFFFF5CFFBF00900FFFFF5CFFCF046
:100D4000010E0001FD6F0E0E56EC00F0050186A1AC
:100D500012D0870EF66E0A0EF76E0900FFFFF5CF70
:100D6000FBF00900FFFFF5CFFCF00001FD6B0C0E5E
:100D700056EC00F011D06F0EF66E0A0EF76E0900F9
:100D8000FFFFF5CFFBF00900FFFFF5CFFCF00001FE
:100D9000FD6B0C0E56EC00F01200FFFFA5D7FFFF15
:100DA000730EF66E0A0EF76E0900FFFFF5CFFBF02B
:100DB0000900FFFFF5CFFCF00001FD6B100E56EFB0
:100DC00000F0FFFFEDD7FFFF8EDF770EF66E0A0E05
:100DD000F76E0900FFFFF5CFFBF00900FFFFEAD730
:100DE000FFFFF2D7FFFF790EF66E0A0EF76E0900CD
:100DF000FFFFF5CFFBF00900FFFF0DD0FFFFF3D79A
:100E0000FFFF7B0EF66E0A0EF76E0900FFFFF5CFAF
:100E1000FBF00900FFFFF5CFFCF00001FD6B000EB9
:100E200056EF00F0FFFFEDD7FFFF050189A312D0B9
:100E3000710EF66E0A0EF76E0900FFFFF5CFFBF09C
:100E40000900FFFFF5CFFCF00001FD6B000E56EC32
:100E500000F026D0050189A702D0D7DE21D043DFDC
:100E6000690EF66E0A0EF76E0900FFFFF5CFFBF074
:100E70000900FFFFF5CFFCF00001FD6B100E56ECF2
:100E800000F0030E0001FB6F00EEFCF0DFC0EEFF90
:100E9000E0C0EDFF200EFE6FFF6B1A0EBCEC00F001
:100EA0001200FFFFC2D7FFFF050189A312D0710E08
:100EB000F66E0A0EF76E0900FFFFF5CFFBF0090092
:100EC000FFFFF5CFFCF00001FD6B000E56EC00F0CB
:100ED00057D0050189A702D098DE52D004DF6B0EEF
:100EE000F66E0A0EF76E0900FFFFF5CFFBF0090062
:100EF000FFFFF5CFFCF00001FD6B100E56EC00F08B
:100F00003C0E046E056A066A076AEDC000F0EEC08A
:100F100001F0EFC002F0F0C003F021EC02F0002875
:100F20000001F76F000E0120F86F020EFB6F3C0E00
:100F3000026E036AF7C000F0F8C001F0C8EC02F0DE
:100F400000C0FCF001C0FDF0300EFE6FFF6B1D0E07
:100F5000BCEC00F0020E0001FB6F3C0E026E036A57
:100F6000F7C000F0F8C001F0C8EC02F004C0FCF0DB
:100F700005C0FDF0300EFE6FFF6B1A0EBCEC00F0EA
:100F80001200FFFF91D7FFFFAEDE750EF66E0A0E60
:100F9000F76E0900FFFFF5CFFBF00900FFFF0AD74E
:100FA000FFFF050185A302D00EDF08D0050185A152
:100FB00002D018DF03D0050186B522DF1200FFFF43
:100FC000F0D7FFFF7D0EF66E0A0EF76E0900FFFFE9
:100FD000F5CFFBF00900FFFFF5CFFCF00001FD6B42
:100FE000000E56EC00F080C500F0A50E00240001B4
:100FF000FB6FFC6B080E91D0FFFFE4D7FFFF7F0E65
:10100000F66E0A0EF76E0900FFFFF5CFFBF0090040
:10101000FFFFF5CFFCF00001FD6B000E56EC00F079
:10102000020E0001FB6F7EC5FCF0FD6B200EFE6F13
:10103000010EFF6F070EBCEC00F081C500F0190E29
:1010400000240001FB6FFC6B090E67D0FFFFD7D7B0
:10105000FFFF810EF66E0A0EF76E0900FFFFF5CF57
:10106000FBF00900FFFFF5CFFCF00001FD6B000E67
:1010700056EC00F0030E0001FB6F00EEFCF0DBC04D
:10108000EEFFDCC0EDFF200EFE6FFF6B070EBCEC29
:1010900000F082C500F0900E00240001FB6FFC6B95
:1010A000090E3BD0FFFFD5D7FFFF830EF66E0A0E69
:1010B000F76E0900FFFFF5CFFBF00900FFFFF5CF4A
:1010C000FCF00001FD6B000E56EC00F0030E000179
:1010D000FB6F00EEFCF0DDC0EEFFDEC0EDFF200E8A
:1010E000FE6F010EFF6F040EBCEC00F0030E00015A
:1010F000FB6F00EEFCF0DBC0EEFFDCC0EDFF200E6E
:10110000FE6FFF6B0B0EBCEC00F083C500F0E70E2A
:1011100000240001FB6FFC6B090EFC234ED6FFFF81
:10112000C4D7FFFF010EE8CF79F505017B6B1200F4
:10113000FFFFF8D7FFFF05017B2B030E7B6503D074
:101140007B6B0501796B0501899B1200FFFFF3D7CB
:10115000FFFF05017B530BE10A0E05017C6103D003
:10116000010E7C2B97D00A0EE8CF7CF515D07BC5FD
:1011700000F0000414E10001010EE05D2C0ED8B473
:10118000DF5D05E20A0EDF27000EE02383D00001B9
:101190002C0EDF6F010EE06F0501899B7BD03C0EAA
:1011A000046E056A066A076AF1C000F0F2C001F039
:1011B000F3C002F0F4C003F021EC02F000C0F3FF32
:1011C00001C0F4FF3C0E026E036AF3CF00F0F4CFCF
:1011D00001F0C8EC02F00450D96E3C0E026E036AB6
:1011E000F3CF00F0F4CF01F0C8EC02F000C0F6FF3E
:1011F00001C0F7FF7BC5E8FF020A08E1170ED960BE
:1012000002D0D92A15D0170ED96E10D07BC5E8FFB1
:10121000030A0EE1000EF75C3B0ED8B4F65C03E265
:10122000F64AF72A05D03B0EF66EF76A0501899B50
:101230003C0E046E056A066A076AD9CF00F0016A9F
:10124000026A036AB8EC11F000C0F7F001C0F8F0D0
:1012500002C0F9F003C0FAF0F6CF00F0F7CF01F0CA
:10126000026A036A0001F7510026F8510122F95180
:101270000222FA5103223C0E046E056A066A076ACE
:10128000B8EC11F000C0F1F001C0F2F002C0F3F0D0
:1012900003C0F4F005017089050189BB03D0040E79
:1012A0002FEC11F01200FFFF54D7FFFF05017B5315
:1012B0000AE1010E05017C6502D07C0792D0010E87
:1012C000E8CF7CF515D07BC500F0000414E10001E7
:1012D000000EE05D1F0ED8B4DF5D05E3F60EDF27DC
:1012E000FF0EE0237ED000011E0EDF6F000EE06BCC
:1012F0000501899B76D03C0E046E056A066A076A72
:10130000F1C000F0F2C001F0F3C002F0F4C003F04D
:1013100021EC02F000C0F3FF01C0F4FF3C0E026EAE
:10132000036AF3CF00F0F4CF01F0C8EC02F00450F0
:10133000D96E3C0E026E036AF3CF00F0F4CF01F0D9
:10134000C8EC02F000C0F6FF01C0F7FF7BC5E8FF64
:10135000020A06E1D95002E0D90611D0D96A0DD0AF
:101360007BC5E8FF030A0BE1F750F61004E0FF0E1F
:10137000F606F72204D0F66AF76A0501899B3C0E4F
:10138000046E056A066A076AD9CF00F0016A026A2C
:10139000036AB8EC11F000C0F7F001C0F8F002C029
:1013A000F9F003C0FAF0F6CF00F0F7CF01F0026ACF
:1013B000036A0001F7510026F8510122F951022277
:1013C000FA5103223C0E046E056A066A076AB8ECFD
:1013D00011F000C0F1F001C0F2F002C0F3F003C060
:1013E000F4F005017089050189BB03D0040E2FECD0
:1013F00011F01200FFFF5AD7FFFF006A700E016E56
:10140000420E026E00C0F7F001C0F8F002C0F9F021
:101410007CC500F0E5EC12F0F7C003F0F8C004F072
:10142000F9C005F0FCEC11F000C0E7F001C0E8F0F5
:1014300002C0E9F0DBC000F0DCC001F0002A000EC1
:10144000012210EC13F000C0EAF001C0EBF002C082
:10145000ECF0DBC0E5F0DCC0E6F000EED5F0EE6AC3
:10146000EE6A00EED7F0EE6AEE6A020EE8CF79F58A
:1014700005018683DAD0FFFFC0D7FFFF05018993FE
:10148000898700012C0EE16F010EE26F1200FFFF51
:10149000F5D7FFFF060EE8CF79F5190EE8CF7EF5F8
:1014A0001200FFFFF7D7FFFF280E05017E6103D072
:1014B000010E7E2B05D0280EE8CF7EF50501899B15
:1014C000050170891200FFFFEFD7FFFF0A0E05012B
:1014D0007E6503D0010E7E0705D00A0EE8CF7EF5AB
:1014E0000501899B050170891200FFFFEFD7FFFFFF
:1014F000070EE8CF79F50A0E2FEC11F0050186836F
:10150000050E2FEC11F00001C80EE36FE46B070E1F
:101510002FEF11F0FFFFECD7FFFF0001010EDE5DA2
:10152000500ED8B4DD5D04E2DD2B000EDE2307D0C3
:101530000001500EDD6F010EDE6F0501899B050174
:101540007089050189BB03D0090E2FEC11F0120040
:10155000FFFFE3D7FFFF0001000EDE5DB10ED8B440
:10156000DD5D04E3DD07000EDE5B07D00001B00E99
:10157000DD6F000EDE6B0501899B05017089050199
:1015800089BB03D0090E2FEC11F01200FFFFE3D747
:10159000FFFF0B0E2FEC11F0050186938691050ECF
:1015A0002FEC11F0050EE8CF79F51200FFFFF1D70F
:1015B000FFFF0501020E891B1200FFFFFAD7FFFF94
:1015C000050189A30DD00501796B050186938691EC
:1015D0000501899F050E2FEC11F0050189930DD0AF
:1015E00000EED5F0EE6AEE6A00EED7F0EE6AEE6A33
:1015F00005018681050E2FEC11F01200FFFFE0D7E8
:10160000FFFF050189A303D00501899305D00501DA
:101610008691050E2FEC11F01200FFFFF2D7FFFFAD
:101620000501796B050186938691050E2FEF11F068
:10163000FFFFF6D7FFFF080E2FEC11F0050EE8CFE5
:1016400079F51200FFFFF7D7FFFF05018693050E1E
:101650002FEC11F0020E0001F76FF86BF40EF96F2A
:10166000010EFA6FF40EFB6F010EFC6F47EC05F0F4
:1016700000EED5F0EE6AEE6A00EED7F0EE6AEE6AA2
:10168000050186978699DBC0E5F0DCC0E6F0120024
:10169000FFFFDBD7FFFF100ED96E180EE16E0E8034
:1016A000E96A0F0E8A16D950F00B8A12E1CF00F0CA
:1016B000040E00168050040B0018D8A40E90D89089
:1016C000D936D890E132E92A030EE964EAD7D890F6
:1016D0000EB0D8801200FFFFDED7FFFF100ED96ECC
:1016E0000E92E16A0F0E8A16D950F00B8A1280B45E
:1016F0000E82D890D936E12A030EE164F3D7D89050
:101700000EB2D8801200FFFFE9D7FFFF0501795321
:1017100018E105016B2B05017F5304E07FC5E8FF4D
:10172000160A02E1630E01D0130E05016B6503D0AA
:101730006B6B05017F2B270E05017F658DD07F6BBD
:101740008BD079C5E8FF050A1CE105016C2B05016A
:10175000805308E080C5E8FF220A04E080C5E8FF66
:10176000420A02E1630E01D0130E05016C6503D03D
:101770006C6B0501802B500E050180656DD0806B70
:101780006BD079C5E8FF060A24E105016D2B050140
:10179000815310E081C5E8FF1E0A0CE081C5E8FF17
:1017A0003E0A08E081C5E8FF560A04E081C5E8FF6B
:1017B000660A02E1630E01D0130E05016D6503D0C8
:1017C0006D6B0501812B650E0501816545D0816B2F
:1017D00043D079C5E8FF070A18E105016E2B050122
:1017E000825304E082C5E8FF2B0A02E1630E01D0B8
:1017F000130E05016E6503D06E6B0501822B460E3C
:101800000501826529D0826B27D079C5E8FF080AD7
:1018100023E105016F2B0501835310E083C5E8FF29
:101820001E0A0CE083C5E8FF3E0A08E083C5E8FF16
:101830005B0A04E083C5E8FF6B0A02E1630E01D096
:10184000130E05016F6503D06F6B0501832B6A0EC4
:101850000501836501D0836B1200FFFF57D7FFFF9F
:10186000050185A72AD00001D52B000ED623010E35
:10187000D65D2D0ED8B4D55D26E3DBC000F0DCC00C
:1018800001F0E5C0E8FF005C026EE6C0E8FF015829
:10189000036E0350800A800F030ED8B4025C05016A
:1018A00002E2868701D0869700EED5F0EE6AEE6AF6
:1018B000DBC0E5F0DCC0E6F006D000EED5F0EE6A65
:1018C000EE6A05018697E3C000F0E4C001F0F10E76
:1018D0000024026EFF0E0120036EDBC000F0DCC0AE
:1018E00001F00350015C02E10250005C10E20001D3
:1018F000D72B000ED823D85DB50ED8B4D75D0DE335
:10190000B40ED76F000ED86B0501868906D000EEA5
:10191000D7F0EE6AEE6A05018699050186A705D023
:10192000050186A902D0050186851200FFFF98D720
:10193000FFFFA4EC12F0BBEC01F0F3EC01F045EC7E
:1019400000F0A8DE03E3050EE8CF79F5C6DEFEE27F
:10195000F28E020E2FEC11F043EC11F052EC10F06D
:1019600065EC11F0050188A722D105018897FFD009
:1019700018D1DFC002F0E0C003F0DBC000F0DCC033
:1019800001F00350015C02E10250005C1CE3F1C075
:10199000EDF0F2C0EEF0F3C0EFF0F4C0F0F0DFC015
:1019A000E3F0E0C0E4F0DBC0E5F0DCC0E6F000EE20
:1019B000D5F0EE6AEE6A00EED7F0EE6AEE6A030E3C
:1019C000E8CF79F5B3D0EAC000F0EBC001F0ECC08D
:1019D00002F07EEC12F0DFC002F0E0C003F0035032
:1019E000015C02E10250005C0AE2E7C003F0E8C0DB
:1019F00004F0E9C005F000EEEAF020EC13F0EAC0D4
:101A000000F0EBC001F0ECC002F07EEC12F000C080
:101A1000E3F001C0E4F0070E2FEC11F00001000E1E
:101A2000DC5D500ED8B4DB5D0FE3050189BF0CD03F
:101A30000501898F0501868100EED5F0EE6AEE6A18
:101A400000EED7F0EE6AEE6A05018683050E2FECF4
:101A500011F06CD00001ED51EE11EF11F0110CE11D
:101A6000040EE8CF79F50501869386910501899FDB
:101A7000050E2FEC11F05AD00001ED07000EEE5BC1
:101A8000EF5BF05B070E2FEC11F00001000EDC5D48
:101A9000500ED8B4DB5D0FE3050189BF0CD0050102
:101AA000898F0501868100EED5F0EE6AEE6A00EEC0
:101AB000D7F0EE6AEE6A05018683050E2FEC11F071
:101AC00035D0050186938691050E2FEC11F0030E9B
:101AD0000001F76FF86BC80EF96FFA6B640EFB6FBD
:101AE000FC6B47EC05F022D005018683050E2FEC38
:101AF00011F00001000EDC5DC80ED8B4DB5D16E30A
:101B0000080EE8CF79F5010E0001F76FF86BE80ECB
:101B1000F96F030EFA6F010EFB6FFC6B47EC05F0DB
:101B200005D005018683050E2FEC11F0050185B364
:101B300006D0050185B103D0050186A532D0090E76
:101B4000E8CF79F52ED0050186938691050E2FEC0E
:101B500011F0030E0001F76FF86BE80EF96F030E3A
:101B6000FA6F640EFB6FFC6B47EC05F01AD079C579
:101B7000E8FF000A01E1FCD6010A01E1F9D6030AF7
:101B800001E1F7D6010A01E165D7070A9AE0010AE7
:101B9000AAE0030AA8E0010AA7E00F0AC2E0010ACE
:101BA000D2E0030E2FEC11F0060E2FEC11F0050120
:101BB00070A34CD00501709370A50FD005017095EE
:101BC000020E0001F76FF86B280EF96FFA6B280E02
:101BD000FB6FFC6B47EC05F00FD0050189BB0CD007
:101BE000010E0001F76FF86B140EF96FFA6B140E0B
:101BF000FB6FFC6B47EC05F079C500F0016AD890EB
:101C000000360136D8900036013684C5E8FF00243E
:101C1000026E000E0120036ED8900234006E033471
:101C2000016E0050800FF66E0150F76E060EF7221F
:101C30000900FFFFF5CF00F00900FFFFF5CF01F02D
:101C400000C0F6FF01C0F7FF28EC13F0050189A5DD
:101C500083D60501899579C500F0D8900034006ECF
:101C6000016A01360050D00FF66E0150F76E060E75
:101C7000F7220900FFFFF5CF00F00900FFFFF5CFC5
:101C800001F000C0F6FF01C0F7FF28EC13F03DDDC6
:101C90000001E151E21103E1050189975DD60001E0
:101CA000E107000EE25B58D6FFFFF2B4F2AA56D16C
:101CB000F294080ED66E0001F507FF0EF623F551DB
:101CC000F6110AE1050188870001E80EF56F030EA1
:101CD000F66F0501080E701B0001F651010AF40EA3
:101CE000D8B4F51903E10501080E701B0501672F33
:101CF00005D00A0EE8CF67F5050189850001D351AB
:101D0000D41104E18A820501889123D00001CF51CA
:101D1000D0110CE08A92CF07FF0ED023CF51D01103
:101D200018E1CDC0D1F0CEC0D2F013D00001D15116
:101D3000D2110FE08A82D107FF0ED223D151D211E6
:101D400008E1CBC0CFF0CCC0D0F00001D307000E2B
:101D5000D45B05017D530CE07D2F0AD0050174533F
:101D600002E0740703D01D0EE8CF74F505018991D8
:101D7000F5C5E8FF200A13E10501F56B8A960F0E01
:101D80008A16800ED96E8A8E8A848A940F0E8A16DD
:101D9000D96A8A508A848A940501709155D0F5C514
:101DA000E8FF100A14E1050170B111D08A960F0EF8
:101DB0008A16C00ED96E8A128A848A940F0E8A16E9
:101DC000D96A8A508A848A94050170813DD08A86B6
:101DD000F5C5E8FF15EED1F0E126000EE222E7504E
:101DE000D96E7F0ED9641BD0F5C5E8FF15EED1F092
:101DF000E126000EE222E750006E00C002F0036A06
:101E00000250000FF66E0350F76E060EF722800E9A
:101E1000F626FF0EF7220800FFFFF550D96E0F0ED1
:101E20008A16D950F00BE16EE1508A128A848A94A6
:101E30000F0E8A16D938F00BF00BE16EE1508A12C2
:101E40008A848A940501F52B0F0E8A1675C5E8FF62
:101E5000F00B8A1280A43AD075C5E8FF050176150B
:101E600011E1050170B306D06AC584F505017083E0
:101E70000501899B0501708B709D0001D00ED96F03
:101E8000070E1ED0050170AD1CD00501708F70B318
:101E900010D0050170A90DD06AC584F505017083C5
:101EA000050189BB02D00501708584C587F5050150
:101EB000898B0501709D708B0001640ED96F000E37
:101EC000DA6F75C5E8FF0501761311D075C5E8FF17
:101ED0000501761507E0050189BB04D00501709B5B
:101EE000709D709F75C5E8FFFF0A05017617050113
:101EF00089AB19D0050170AD16D00501708F70B394
:101F000009D087C584F505017083050189BB02D01E
:101F1000050170850501898B0501709D708B00019D
:101F2000640ED96FDA6B15EE75F0D890E7360501BF
:101F30006A2B030E6A6504D06A6B100EE8CF75F544
:101F4000050170AB0BD00001D951DA1103E1050195
:101F5000708D709B0001D907000EDA5B9EBA9DAAB6
:101F600018D0ABA403D0AECF8AF513D0AECF8AF58C
:101F70000501712B130E716501D0716B71C5E8FFFE
:101F800015EE8BF0E126000EE2228AC5E7FF05017F
:101F900089899EB89DA816D069C5E8FF0501721908
:101FA00010E069C5E8FF15EE9FF0E126000EE22281
:101FB000E750AD6E0501692B130E696503D0696B9F
:101FC00001D09D98F6C5F5FFF7C5F6FFF8C5F7FFF8
:101FD000F9C500F0FAC502F0FBC503F0FCC5DAFF55
:101FE000FDC5D9FFFEC5E2FFFFC5E1FF1100FFFF00
:101FF0005CD6FFFFE1CFFFF5E2CFFEF5D9CFFDF5CF
:10200000DACFFCF503C0FBF502C0FAF500C0F9F524
:10201000F7CFF8F5F6CFF7F5F5CFF6F545D6FFFF94
:10202000D96EF29E72C5E8FF05EE9FF0E926000E1C
:10203000EA22D9CFEFFF0501722B130E726501D092
:10204000726BACA20FD069C5E8FF05EE9FF0E926E0
:10205000000EEA22EF50AD6E0501692B130E696583
:1020600001D0696B9D88F28E1200FFFFD9D7FFFF68
:10207000F29E0501682B130E686501D0686B71C56F
:10208000E8FF0501686302D005018999F28E68C5F1
:10209000E8FF05EE8BF0E926000EEA22EF50120071
:1020A000FFFFE6D7FFFF050189A94ED0E0DFE8CFAB
:1020B000F3F5F3C500F00028050103E1040E7A1BD7
:1020C00010D07AA50ED005017A817A937A95210EE7
:1020D000E8CFF2F50501F16B0001AA0EA76F000E23
:1020E000A86F05017AB530D005017AA11CD0050191
:1020F000F207F2290EE0F2C5E8FF1E0A14E11E0EF7
:102100000501F36503D005017A910DD0F3C5F2F511
:102110000AD005017A917A83F3C5E8FF0501F163DE
:1021200002D005017A8705017AB30ED0A7C0E9FF76
:10213000A8C0EAFFF3C5EFFF0001A72B000EA823FC
:10214000F3C5E8FF0501F1271200FFFFACD7FFFF41
:10215000F36EE16A010EE8CFAAF0F3CFABF02ED018
:10216000070EE8CFACF07CC5AFF0DFC0ADF0E0C04B
:10217000AEF0F1C0B0F0F2C0B1F0F3C0B2F0F4C014
:10218000B3F02DD0010EE8CFACF086C5ADF027D06E
:10219000020EE8CFACF0E3C0ADF0E4C0AEF01FD06B
:1021A000010EE8CFACF07EC5ADF019D0020EE8CF3D
:1021B000ACF0DDC0ADF0DEC0AEF011D0ABC0E8FFDA
:1021C000040ACEE0010ADEE0020AE2E00F0AE8E0DB
:1021D000010AECE0020AEAE00001AC6BAD6BFF0E15
:1021E0001EDFAAC0E8FF1BDFABC0E8FF18DFACC0F2
:1021F000E8FF15DFAAC0E8FFE126ABC0E8FFE12653
:10220000ACC0E8FFE126F36AACC0E8FFF35C1EE275
:10221000F35000EEADF0E926000EEA22EF50E12681
:10222000F35000EEADF0E926000EEA22EF50F7DEA3
:10223000F35000EEADF0E926000EEA22EF50006EFA
:10224000002802E1FF0EEBDEF32ADED7E150E7DEE5
:10225000E12802E1FF0EE3DE1200FFFF79D7FFFF66
:10226000D96E73C5E8FF05EEB3F0E926000EEA2249
:10227000D9CFEFFF0501732B1D0E736501D0736B72
:102280001200FFFFEDD7FFFF050189B11BD073C519
:10229000E8FF0501741916E00501898174C5E8FF9E
:1022A00005EEB3F0E926000EEA22EF5050DFF29E71
:1022B0000501742B1D0E746501D0746BF28EC80E6F
:1022C000E8CF7DF51200FFFFDFD7FFFF05017AA7FA
:1022D0004CD005017A97AAC000F0000446E135D041
:1022E000ACC0E8FF030A3DE1AEC077F5AFC078F5BA
:1022F00038D0ACC0E8FF070A34E1ADC0DFF0AEC0B3
:10230000E0F0AFC07CF5B0C0F1F0B1C0F2F0B2C007
:10231000F3F0B3C0F4F025D0ACC000F0000421E12C
:10232000ADC085F51ED0ACC0E8FF020A1AE1ADC011
:10233000DBF0AEC0DCF015D0ACC0E8FF020A11E162
:10234000ADC0DDF0AEC0DEF00CD0ABC0E8FF010ADE
:10235000C7E0030ACEE0010ADFE0050AE4E00C0A68
:10236000EBE00501899105017D6B1200FFFFAED7FF
:10237000E96AEA6A0050086E0150096E02500A6E5E
:1023800003500B6E026A036A08500402F3CF00F098
:10239000F4CF01F008500502F3500126F450022258
:1023A00009500402F3500126F4500222D8B0032A47
:1023B00008500602F3500226F45003220950050289
:1023C000F3500226F45003220A500402F35002266E
:1023D000F450032208500702F35003260950060266
:1023E000F35003260A500502F35003260B50040253
:1023F000F3500326EEEF12F0E96AEA6A7CEC02F091
:1024000089EC02F0096A0A6A0B6A0E9A0EB60E8A05
:10241000065203E0075002E10E881200065E770EB6
:1024200004E30626D8B00E8403D00626D8A00E8674
:102430000830081A180E056ED89009360A360B3681
:10244000026606D00450015C02E10350005C07E321
:102450000350005E0450015AD8A002060980D890AB
:10246000003601360236052EE7D70950006E0A50B5
:10247000016E0B50026EA4EF02F00650075C0AE3F7
:10248000D8B41200D890023201320032062A065027
:10249000075CF6D7D890053204320332072A06507B
:1024A0000718D8B41200F6D7800E051AE96AEA6A4E
:1024B0007CEC02F089EC02F0E0DF08B017D808A24B
:1024C00007D0031E041E051E000E032A0422052247
:1024D000035000260450012205500222086A02AE71
:1024E000A4EF02F003D80880A4EF02F0001E011E42
:1024F000021E000E002A012202221200E96AEA6A84
:102500007CEC02F0036A820E062606BE85EF02F01E
:10251000F00E062606BE11D0180E065C02E385EF0B
:1025200002F0065204E108B014EC13F012000606A3
:102530000036013602360336F4D7D8900232013223
:102540000032063EFAD7EFD7FFFFF80E806E8168A3
:10255000F90E826E3D0E926E936AD80E946E070E3F
:10256000C16E010EC26EC40ED56E080ED66E200E60
:10257000AC6E900EAB6E330EAF6EF294F28A9D8A03
:10258000F28C1200FFFFE1D703AE04D0088014ECF8
:1025900013F001D0086A8E0E066EE96AEA6A0352E9
:1025A000D8B4A4EF02F0D8900332023201320032E4
:1025B000062AF5D7016A026A036A00AECAEF12F072
:1025C000010602060306C4EF12F0016A026A036AFA
:1025D000CAEF12F0036A026A016A006AE950EA105F
:1025E00008E003C0EDFF02C0EDFF01C0EDFF00C039
:1025F000EFFF000C02500002F3CF04F0F4CF05F01F
:1026000002500102F350052603500002F350052644
:102610001200026A01BE02060250036EC4EF12F0FD
:10262000026A036ACAEF12F0001E011E021E031E98
:10263000000E002A0122022203221200800E051A37
:10264000EECF00F0EECF01F0EFCF02F058EF12F036
:10265000FA6E0500F850FF6EF750FE6EF650FD6EF4
:04266000FA5012001A
:020000040030CA
:04000000FFFEF6FE0B
:02000600FBFFFE
:00000001FF
